:1000000000EEFCF0EE6AEE6AEE6AEE6A02EEFFF0D7
:06001000EE6AAAEF1FF0EA
:103F3800FC000001FF0EFC07FD23FE23FF23FF51B9
:103F4800FC11FD11FE11D8B41200F3D7B8EC1FF024
:103F5800C4EC1FF0E8CFFFF2FFC2E8FFC0EC1FF08F
:103F68002A0EC0EC1FF0F4D7240EAC6E900EAB6E88
:103F78007E6A810EAF6E1200ACA2FED7AD6E120043
:103F88009EAAFED7AE5012009EAA000CAE50120098
:103F9800FC00D96AD9500001FC25006E000EFD21F5
:103FA800016E00C0F6FF01C0F7FF020EF76403D0F0
:103FB8000800F55005D0F6CFE9FFF7CFEAFFEF503C
:103FC8000009D8B41200D9500001FC25006E000E7B
:103FD800FD21016E00C0F6FF01C0F7FF020EF76475
:103FE80003D00800F55005D0F6CFE9FFF7CFEAFF78
:083FF800EF50C2DFD92ACED739
:020000040030CA
:0A000000FF32F9FEFFFBBFFFFFFF18
:00000001FF
